:030000000219FDE5
:03000B000200A848
:03002B000201636C
:03005B000202EDB1
:030073000202D3B3
:1000800002030406080C10182030406080040608A3
:100090000C10182030406080A0C000070F1F3F05E3
:1000A000050D050305030302C2AFC0D0C0E0206206
:1000B00017E5256002E473E525F4F58A758B00D217
:1000C00062D0E0D0D0D2AF3285268AC262E526F473
:1000D0006035306803207210758B00D0E0D0D0C23C
:1000E00093C295C297D2AF32C293C295C297206E87
:1000F0000C206609740AD5E0FDE57E4290758B0000
:10010000D0E0D0D0D2AF32758A00C28DD26201FD6C
:1001100001B7306805206602D29301B73068052028
:100120006602D29501B7306805206602D29701B702
:10013000C29230680A2066077408D5E0FDD29301A8
:10014000B7C29430680A2066077408D5E0FDD295DE
:1001500001B7C29630680A2066077408D5E0FDD260
:100160009701B7C2AFC2AD53E6EFC0D0C0E0D2D363
:10017000D2AFC2CEE52A6007207449152A21C4787F
:1001800000790020742EE580307E01F430E302789F
:10019000FF53DACF207E0343DA20307E0343DA10A8
:1001A000C2D8C271E580307E01F430E30279FFC32A
:1001B000E89970CB306103752A18207403752A18EA
:1001C000885FD27020740DE52B6004152B21D44379
:1001D000DA01C2D82070024136A85F206102C270E5
:1001E000207431C3E894F0400374F0F8E8C4540F6D
:1001F00028F87984B703024114C313C3138721205D
:100200000802C313200A06C3C898F8411428F850FE
:100210000374FFF8C3E895685003E568F88822E5A1
:100220002D54066011E533C313C31324062522F5AC
:100230002250037522FF852224A824C3E524956457
:100240004002A8648825E5697002417AC3E8AA697A
:100250009A5003E8FAE4F9EAC333FBE56BF45B294F
:10026000400D256AF8E56A6002156A400B417A0A7A
:10027000C3E56A9A5002056A78FF8826C26EC3E514
:100280002694F84002D26EC3E52594404002D26421
:1002900020CF0AD0E0D0D043E610D2AD32C2CF0595
:1002A0003A7801E52A6005307402152AC3E55F94A7
:1002B00001400575620041C9756300756C00E56217
:1002C0002401F56250037562FFD0E0D0D043E61000
:1002D000D2AD32C2AFC0D053E67FC2607591008507
:1002E0005694855795759104D0D0D2AF32C2AF5392
:1002F000E6EFC2ADC0D0C0E0C0F0D2D3D2AFA8FB11
:10030000A9FCC2D8307102615453DACF207E034376
:10031000DA10307E0343DA20D271E580307E01F4BA
:1003200020E302612B88278928A17B53DACF207E26
:100330000343DA20307E0343DA10C2D8C27130742E
:1003400002A1677800E580307E01F430E302A16706
:10035000885FA14F53DACF207E0343DA20307E033B
:1003600043DA10C271206102812D53DACF207E035F
:1003700043DA10307E0343DA20C2D8D271885A891A
:100380005BC3E89558F8E99559F97B007E087A0037
:10039000C3E8948CE994005005755E00811F8821A4
:1003A00078A2E6A8216055C3E894C8E994005008F3
:1003B000E4D2E4FB7A0A61FAC3E89468E994015054
:1003C00008E4D2E3FB7A0F61FAC3E894D0E994021F
:1003D0005008E4D2E2FB7A1E61FAC3E894A0E994E3
:1003E000055008E4D2E1FB7A3C61FAC3E89498E94D
:1003F00094085008E4D2E0FB7A787E00C3E8955C6C
:10040000FCE9955DFD30E70AECF42401FCEDF434E1
:1004100000FD755E00C3EC9AED9E5003755E018889
:100420005C895D855A58855B597802A14FC3E89570
:1004300027F8E99528F9307C02A133307B02A133FB
:10044000307A02A12C2075028150E9FDE8FC816F11
:10045000E9C313F9E813F8307902A12CE9C313F9C1
:10046000E813F8307802A12CE9C313FDE813FC204F
:0E0470006126C3EC941CED940240028186EDDF
:10047E007018C3EC94C850120529C3E529940A508C
:10048E0002A167755F00D270A167E5296002152988
:10049E007888E6F97400207F087896B90302789E72
:1004AE00E624FAFEE43400FFC3EC9EFCED9FFD92C1
:1004BE0008B90310A2085007207609D27681D230EF
:1004CE007602C276A2085016B9030DECF42401FC94
:1004DE00EDF43400FD0204EC78007900A133B90389
:1004EE0015EC33FCED33FDC3EC940AFCED9400FDEA
:1004FE0050047C007D00C3EC94FFED940040067820
:10050E00FF7900A133EC8575F0A4C5F0A2F733F89E
:10051E007900400302054F78FF790002054FE9C3C9
:10052E0013F9E813F8307C0EE9600278FFC3E81384
:10053E0038F8E43400F9C3E894FFE99400400278F7
:10054E00FF885FD270206102A167741FF4552F4B94
:10055E00F52FC274EB7002D274752A1830740375BD
:10056E002A0A306102A17B20740353DAFE20740341
:10057E00752B06D0F0D0E0D0D0D2AD43E610327954
:10058E00010205AB79030205AB790A0205AB791EB0
:10059E000205AB79640205AB79C80205AB7817E4A6
:1005AE00D5E0FDD8FAD9F6227A147B780205D27AF4
:1005BE00107B8C0205D27A0D7BB40205D27A0B7BAE
:1005CE00C80205D27902B27DE4C294D5E0FDD2957F
:1005DE00D5E0FDC295D5E0FDD294D5E0FDD293E5F0
:1005EE0076D5E0FDC2937496D5E0FDD9D9EAF8D55B
:1005FE00E0FDD8FBDBCEC29422C37C007D0075F0FB
:10060E000005F0EA33FAEB33FB50F6EB13FBEA137B
:10061E00FAC3E9FFE8FEE89AF8E99BF95004EFF90E
:10062E00EEF8B3EC33FCED33FDD5F0DFEDF9ECF87D
:10063E0022E889F08A20D2D4F8A9F07B0030F70B9B
:10064E007BFFF42401F8E9F43400F9E88520F0A4E6
:10065E00ADF0F8E98520F0A4AFF0FEED2EF97400B0
:10066E003FFA7C04C3EA13FAE913F9E813F8DCF451
:10067E008BF030F70AE8F42401F8E9F43400F9E8D5
:10068E0089F0C2D4F8A9F02222C3E54113F9E5405E
:10069E0013F8C3E54598F8E54699F9500CC3E8946C
:1006AE0080E994FF40160206CEC3E8947FE99400D9
:1006BE0050030206CE787F79000206CE788079FF4D
:1006CE00884A894B22E54A2547F8E54B3548F98596
:1006DE004B20E4300701F43549FA30E709C3EA94B8
:1006EE00F0401502070CC3EA940F500302070C7872
:1006FE00FF79FF7A0F02070C780079007AF0C3E5D4
:10070E00249564500AC374019524500B02072AE500
:10071E004B20E70E02072AE54B30E706884789484B
:10072E008A492278A4E6FAC3E54A33F8E54B33F951
:10073E00D13FE930E70BC3E89480E994FF4013E121
:10074E0064C3E8947FE994005002E164787F7900F5
:10075E00E164788079FFE820E715C3E52398F84037
:10076E0009C3E89401400302078B780102078BE866
:10077E00F424012523F8400302078B78FF884C22CE
:10078E0078A5E6FAA848A949D13FE930E70CC3E8B5
:10079E009401E994FF40160207BFC3E894FFE99461
:1007AE000050030207BF78FF79000207BF78017976
:1007BE00FFE920E715C3E54C98F84009C3E894011A
:1007CE0040030207E678010207E6E8F42401254C0F
:1007DE00F840030207E678FF88242278FFC26420DF
:1007EE00693D206A12D264C3E541940A4009C3E50B
:1007FE002594405002C26479A1E76023E541601F51
:10080E0074FF8541F0848539F0306A0375F005A4D4
:10081E00F8C5F0600278FFC3E895675002A86788B4
:10082E006622C3E5409440E5419401E56650031409
:10083E000141046002F566220208492275E8902201
:10084E007883E6FFE5E820ECF7A8BDA9BE0573C3E3
:10085E00E57394084052757300E9FA79A0E7604495
:0E086E00EA7007E574601B020884C3E8957405
:10087C006010E5745006600C140208900460F902D4
:10088C000890E574F574C394A8401B7564C0C394B8
:10089C00054013756480C39405400B756440C39484
:1008AC0005400375640075BB0122E564F460020524
:1008BC0064E573B4070375BB1E22743279A687F006
:1008CC00A4C5F0A2F733F8C3E895644002A8648885
:1008DC00228824882588268867227540007541F077
:1008EC0022C2AF75C820A8CCA9CDAA3A30CF010A34
:1008FC0075C824D2AFAB3BAC3C883B893CC3E89B6E
:10090C00F8E99C206908F93067024102215FAD3D8E
:10091C008A3DF9EA9DFA600478FF79FFAE3EAF3F5D
:10092C008B3E8C3FC3EC9FFCC3E99CF542A83BA9D2
:10093C003CC3E89EF8E99FF9C3E54113FBE540137E
:10094C00FAE82AF540E93BF54150067540FF754140
:10095C00FF21A9AA40AB41AC40AD417E047F02C34C
:10096C00EB940440021E1FC3EB940840021E1FC3ED
:10097C00ED13FDEC13FCDEF7C3EA9CFAEB9DFBEFE9
:10098C006009C3E913F9E813F8DFF7EA28FAEB3941
:10099C00FB8A408B4150067BFF8B408B41C3EB9411
:1009AC00025002D2673069047F0321D47892E6FFAB
:1009BC00C3E537948240110FC3E53794A040010F73
:1009CC00C3EF940640027F057E05E541C4540FF940
:1009DC00E541C454F0F8E540C4540F28F8C3E89E30
:1009EC00FAE99400FB4009C3EA9402EB940050042A
:1009FC007A02E4FB414EAA40AB41EBC4FEEAC4547C
:100A0C000F4EFCC3EA9CFAEB9400FBC3E813C31330
:100A1C00F8EA28FAEB3400FB8A408B41C3EB9402D2
:100A2C004002C2677805EBC4FE7B00EAC4540F4E4B
:100A3C00FAC3EA98FA4005C3940250027A027892FB
:100A4C00E6FF306002414E855256855357D26043C3
:100A5C00E680C3E49AF8E49BF930670241E8E8FACF
:100A6C00E9FBD3E913FDE813FC88528953C3EF94D7
:100A7C00036038EF20E00DE82CF8E93DF9ECFAEDD5
:100A8C00FB020AA3E828F8E939F9C3E82402F8E9DB
:100A9C003400F97AFE7BFFC3EF9403400E8A548B2B
:100AAC0055884E894F8C508D51611C885489558ABC
:100ABC004E8B4F8C508D51306920C3E533940340DD
:100ACC0019E542A2E713F8E555F4240138400B2050
:100ADC00E7087554FFF42401F555611CE8FAD3E8D6
:100AEC0013FC8852C3EF94036020EF20E007E82C3E
:100AFC00F8ECFA6108E8282402F87AFEC3EF9403B4
:100B0C0040088A54884E8C50611C88548A4E8C50F4
:100B1C00E56BC3335002646BF56B30600261267574
:100B2C003402D26043E680E52D54066026A840A925
:100B3C0041C3E913F9E813F8C2AF53E67F7591008E
:100B4C00C3E498F594E499F595759104D26043E665
:100B5C0080D2AF22D265754400752000306B0375CE
:100B6C002040020B7FD265754400752040306B032A
:100B7C00752000D2AF7801206722E52D5406600263
:100B8C00C265C3E54194054013780294054008788A
:100B9C0003940540027806306902780A206019E552
:100BAC0044601530690AC3E53394034003D5340619
:100BBC00D2AFD26C8159712ED2AF0000C2AF206778
:100BCC0026E541C3FB940F40027B0FEB24053073E9
:100BDC000123306A02742820620123F930690279FA
:100BEC0082E58BC39940B50544E59E7005E59B02F3
:100BFC000C00E59A5440B52002814330690A08C3C1
:100C0C00E8940A40010861A8206502617FC265531F
:100C1C00E67F7591003067107594007595FE75919F
:100C2C0004D26043E680617FAE40AF41C3E49EF5E1
:100C3C0094E49FF595812AC3E53394025002617FB9
:100C4C00306502617FD802815761A8C26C53E67F80
:100C5C00759100855494855595759104854E5685EE
:0F0C6C004F57D26043E680D2AFE52D54066008A3
:100C7B00206A020533020C93306C0D206B0A206541
:100C8B00071581158102153A22780030640530650D
:100C9B00027801E53775F007A4F9E5F028F5F0E9DE
:100CAB00A2F013A2F113A2F213F537C394785003F9
:100CBB00753778C3E53795384008D266C293C2952D
:100CCB00C29730600281CD855056855157D2604313
:100CDB00E68022207D14C2AF754302C294D292D219
:100CEB00AF759F33759E00020EBFC2AF754302C234
:100CFB0094D296D2AF759F33759E00020EBF3072A1
:100D0B0043207D20C2AF754303900141757E10C215
:100D1B0097C296306204D295A127D294D2AF759E1A
:100D2B0023020EBFC2AF754303900141757E10C203
:100D3B0093C292306204D295A147D294D2AF759EE2
:100D4B0022020EBF207D17C2AF75430390011CC258
:100D5B0097306202D295D2AF759E23020EBFC2AFFF
:100D6B0075430390011CC293306202D295D2AF75CA
:100D7B009E22020EBF207D11C2AF754304C292D2D8
:100D8B0096D2AF759E22020EBFC2AF754304C296B8
:100D9B00D292D2AF759E23020EBF307249207D23B3
:100DAB00C2AF754305900130757E04C295C2943075
:100DBB006204D293A1C3D292D2AF759F33759E00BA
:100DCB00020EBFC2AF754305900152757E40C295AE
:100DDB00C294306204D297A1E6D296D2AF759F33FC
:100DEB00759E00020EBF207D1AC2AF7543059001A0
:100DFB0012C295306202D293D2AF759F33759E00AB
:100E0B00020EBFC2AF754305900126C2953062E852
:100E1B00D297D2AF759F33759E00020EBF207D1106
:100E2B00C2AF754306C296D294D2AF759E23020E03
:100E3B00BFC2AF754306C292D294D2AF759E220247
:100E4B000EBF307242207D20C2AF7543019001521C
:100E5B00757E40C293C292306204D297C16BD29618
:100E6B00D2AF759E22020EBFC2AF75430190013007
:100E7B00757E04C297C296306204D293C18BD29214
:100E8B00D2AF759E23C1BF207D16C2AF75430190B3
:100E9B000126C293306202D297D2AF759E22C1BF98
:100EAB00C2AF754301900112C297306202D293D246
:100EBB00AF759E23C26622900110757E00C293C24D
:100ECB0095C297C292C294C296C26222788076FF74
:100EDB000876FF0876FF0876FF0876030876040885
:100EEB007607087603087601087601788C76010878
:100EFB0076FF0876FF0876FF0876FF0876FF087600
:100F0B00030876FF0876FF0876FF0876250876D06B
:100F1B000876FA0876FA0876040876FF0876010850
:100F2B00760008767A0876FF08760108760108764F
:100F3B0000087603227887E6FFC272BF0302D272E3
:100F4B007888E6C394036008C27DE630E102D27D67
:100F5B00C27E7889E630E102D27EC3EF940260084C
:100F6B00758E01D273020F78758E00C27322788052
:100F7B00E6149000809378A4F67881E614900080B4
:100F8B009378A5F67886E61490008D9378A6F6787C
:100F9B009CE67538FF75390CB402067538A07539A7
:100FAB000AB4030675388275390578A3E6149000E8
:100FBB009A93F569D1C222227896E6FA7897E6FBE6
:100FCB007888E6B40305C3EB940EFB307F047A00FC
:100FDB007BFFC3EB9AFCC3948250027C8275750035
:100FEB000575EC8575F0A4C3E5F0947D40F222D233
:100FFB007FF1C312059C7A007B007C10120592E5F1
:10100B005F2AFA74003BFBDCF37C04C3EB13FBEAB3
:10101B0013FADCF7FEC27F120FC322E5EF20E603C3
:10102B007520000520903DFFE520146006901FFF02
:10103B001460009304600375EF1253D9BF7581C020
:10104B0043FF8012058D75EF0243B203E5B3240411
:10105B0020E70DF521E5B120E0068521B343B10171
:0F106B00120EC275800875A40075F1FF75D4F7D9
:10107A0075900275A5FC75F2FC75D50075A0FD7515
:10108A00A60275F30275D60075B0FF75A70175F44F
:10109A00FF75E241E4F8F6D8FD756B01120ED7121E
:1010AA00157C78988676753001C2AF1205A61205AE
:1010BA00B612059C1205BD12059C1205C412059CA8
:1010CA001216951205A61205A61205A1C2AF78FA44
:1010DA0079FA308307D9FBD8F7021C00120F4012A5
:1010EA000F79120FC2120FC378988676120EC27544
:1010FA00885075891275C82475910475D84075A8E9
:10110A002275B80275E690759B80759D00759A8068
:10111A00759C0075D10E75BC5875BB0175BA1F75E3
:10112A00E88012058DD2AF12084653DACF207E032B
:10113A0043DA20307E0343DA1043DA01C2D8C2719F
:10114A001205A6D2617B037A0CE55E70077A0CDB86
:10115A00030210D612059C2070030210D6C270E555
:10116A005FC3940240E1E52F541F856160F561B5C4
:10117A0060D5DAD5C26153DACF207E0343DA203054
:10118A007E0343DA10C2D8C27178A2E67008D2741C
:10119A00E52F54E0F52FC2757529001205A13074A8
:1011AA0009C3E529940A4002D275120592780230E1
:1011BA0074027800C3E55F9840F0C2AF1205B61218
:1011CA0005B61205B6D2AF1205A6754D007888E6A7
:1011DA00B4030241BC120592788CE6C39401500311
:1011EA000212BCE530C3940150030212BC207435CC
:1011FA00C3E55F94FF50030212BCC2AF1205CBD203
:10120A00AF1205A1C3E55F940150EFC2AF1205B654
:10121A001205971205B6D2AF1205A1C3E55F94FF76
:10122A0040E902171A7F05D27F120FC31205A1C225
:10123A00AFC27F120FC3AE5FC3E55F947FD2AF40E8
:10124A007B12058DC2AF1205CBD2AFDFDA120FFACD
:10125A00C3EE94057897F61205A61215BE12169DCE
:10126A007F0AD27F120FC31205A1C2AFC27F120F2B
:10127A00C3AE5FC3E55F947FD2AF50E412058DC25F
:10128A00AF1205B61205971205B6D2AFDFD4120F08
:10129A00FAEE24057896F61205A61215BE1216CC99
:1012AA001205A1120FC3C3E55F94FF500221F70292
:1012BA00171AC3E55F954D4003855F4D1205A17866
:1012CA00017988E7B403027805C3E55F98400221F3
:1012DA00D7C2AF1205CB1205CB1205CBD2AF12057E
:1012EA00A6753000E4F531F5320531E531F470398F
:1012FA000532789AE67819146012783214600D78FB
:10130A007D14600878FA146003753200C3E53298D8
:10131A00401715327531B478998676C2AF1205CB6B
:10132A00D2AF789886761205A1120597E52A70053C
:10133A0030740201D678012074027806C3E55F98FA
:10134A0040A77888E6C3940360031205A1E52A70D2
:10135A00030210D6C2AF120EC2E4F522F523F52419
:10136A00F525F526F56AD2AF7885E6C333F568E444
:10137A00F545F546F547F548F549F573F52CF52D8C
:10138A00F53775730875BB1E12058D12084AE5E814
:10139A0020ECFBA8BDA9BEE97001F8887412084EBA
:1013AA0075730875BB1E7887E6FE7602120F4078C1
:1013BA0087EEF6C2AF7564FF1208C68522648522DD
:1013CA0065852266D2AF75220175240175250175DE
:1013DA00260185636C756D017888E6B40307C27DC2
:1013EA00307602D27DD268D269753300120E281285
:1013FA000E4D1208E61208ED1208E61208ED120860
:10140A00E602141BC2AF120F40D2AF75730075BB50
:10141A0001120B71120696120C94120CDE1208EDD0
:10142A00120B60306D031206972067031207E9302A
:10143A006703120830120C94120D091208ED120BF0
:10144A0071306D031206D3120C94120D801208ED3E
:10145A00120B60306D03120731120C94120DA51293
:0E146A0008ED120B71306D0312078E120C94F8
:10147800120E281208ED12084A120B60120C941270
:101488000E4D12084E1208ED306932206B2F856719
:101498006485676585636C756D0179187A0CC3E599
:1014A8003399400CC269D26A8A357564FF0214C543
:1014B800C3E55F9401400302141B021542306A1B06
:1014C800206B18E535147004C26A810EF535C3E542
:1014D8005F9401400302141B021542753600C3E5F0
:1014E800627882985054307404E52A604D7888E612
:1014F800B40317207D05207607A112307602A112C9
:10150800206B07D26B856764815A78F0306B05854C
:1015180067647820C3E541985002811B306B1BC279
:101528006BC27D307602D27DD26A753512856764CA
:10153800811B0536E55F6002A145753600C2AF1212
:101548000EC27887E6FE7602120F407887EEF6E440
:10155800F522F523F524F525F526F568C268D2AFFE
:1015680012058D120EC2307409C3E5369405400287
:1015780001D641EE901A0D7820121600E520B45AD3
:101588000CA3121600E520B4A50302159E120ED76F
:101598001215BE0215BD901A0378807B0A12160038
:1015A800A308DBF9901A0F788C7B18121600A30891
:1015B800DBF9901A2722C2AF12163F121619901A99
:1015C80000740E121605A37404121605A3741412DF
:1015D8001605901A0378807B0A121604A308DBF913
:1015E800901A0F788C7B18121604A308DBF91216D0
:1015F80052121630901A2722E493F622E6438F01FE
:10160800538FFD75EF0275B7A575B7F1F0538FFECF
:1016180022438F02438F0175EF0275B7A575B7F1A5
:10162800901A0DF0538FFC22901A0D745AD1059020
:101638001A0E74A5D105227A3079D07820901A40F4
:10164800D100E520F709A3DAF7227A3079D0901A89
:1016580040E7D10509A3DAF922AB77A878BB0102E4
:101668007984BB02027985BB03027986BB040279BF
:1016780092BB05027987BB060279A3BB0702799C56
:10168800BB08027988BB09027989E8F7227C051230
:1016980005A6DCFB22C2AF1205B61205BD1205C4B1
:1016A8001205CB1205971205B61205BD1205C41214
:1016B80005CB1205971205B61205BD1205C4120511
:1016C800CBD2AF22C2AF1205CB1205C41205BD1290
:1016D80005B61205971205CB1205C41205BD1205F1
:1016E800B61205971205CB1205C41205BD1205B630
:1016F800D2AF22AE77AF78C2AF1205B61205B612D6
:1017080005B6120597DEF21205CB120597DFF8D25F
:10171800AF22D19DD195D1957577017578017579ED
:1017280000D1FB7C05AD5F1205A6C3ED955F70F592
:10173800C3E55F9401400AC3E55F94FF4032021796
:1017480056D161B1BED19DC2AF75EF12D195DCD52E
:101758000579C3E5799403500280C6D1950578E5EB
:10176800771490009F93F808C3E57898500280AEEC
:10177800D195D1950577C3E577940A5002809C12DC
:0B1788000ED7B1BEC2AF75EF12D195B5
:0319FD00021026AF
:101A00000E0414FFFFFFFF0304070301015AA501A1
:101A1000FFFFFFFFFF03FFFFFF25D0FAFA04FF01DE
:081A2000007AFF01010003FF41
:101A400023506C6174696E756D31353041232020EF
:101A500023424C48454C4923463331302320202033
:101A60002020202020202020202020202020202076
:101C0000C2AFC2D353D9BF7581C043B20343FF8073
:101C1000752438752503B1C975EF0275E24043F1AB
:101C20000853A4F775D400D2837DFA780379E67C53
:101C300010752200752300901DD67B0675249875BB
:101C400025013083028142208308D8FBD9F9DCF7D3
:101C500081B4308308D8FBD9F9DCF781B4B189E4C9
:101C600093A3C39A6004DDC381B4DBDBB17B600264
:101C7000812B7B08E493FAA3B15CDBF87A30B15C8A
:101C8000752200752300B17BEAFCEBFDC3ED94FEE9
:101C9000400EB17B8A278B28ED30E0048A828B834B
:101CA000B17B7AC270D8C3ED94FE601350CEBD00F4
:101CB00025EC60097520007521FF0200008100A855
:101CC00027A9280809D804D90281D3B17FEA89AAB3
:101CD000F281C50D81A0C3ED94035049EDA2E092BD
:101CE000007AC5C3E5829400E583941C50902000DF
:101CF00010438F02438F0175B7A575B7F1F030001F
:101D00001FA827A9280809438F01538FFDD804D99C
:101D100002A12089AAE275B7A575B7F1F0A3A10DBC
:101D2000538FFC817C7AC1BD030CE493A3FAB140CC
:101D3000DCF8B138817C817EAA22AB23B15CEBFA5E
:101D4000EA6222752608C3E52313F523E52213F57D
:101D50002250066323A0632201D526EAB1C9B1C986
:101D600075260AEAF4200102D283300102C283B14F
:101D7000C9C3134002C201D526EB22B17FEAFB2082
:101D80008302A17F308302A184752608AE24AF258B
:101D9000C3EF13FFEE13FEB1CDB1C9C3EA13308315
:101DA000024480FA30E703632201C3E52313F523DD
:101DB000E52213F52250066323A0632201D526D91C
:101DC000E52265236523F52222AE24AF250E0FDE22
:101DD000FEDFFCD20122424C48656C693437316326
:041DE000F3100601F5
:00000001FF
